:020000000528D1
:06000A000F308A000327FD
:100010008A01A1011220A000A008031909282E209E
:10002000A10A0A282108820743346F346E346734EA
:1000300072346134743475346C34613474346934BA
:100040006F346E3473342034663472346F346D34EC
:1000500020344134573443340D3400340F308A0097
:10006000200814278A01080083168E309F0083120F
:1000700081309F007D3023278A011F151F193E28DC
:100080001E3084000F308A001A279E3084001A2701
:060090000D301427382892
:02400E00F63F7B
:00000001FF
